 buspcie950

 Timestamp is 494a8a50 (Thu Dec 18 17:37:20 2008)

 Preferred load address is 10000000

 Start         Length     Name                   Class
 0001:00000000 00000a34H .rdata                  CODE
 0001:00000a34 0000005aH .rdata$debug            CODE
 0001:00000a8e 00001e30H .text                   CODE
 0001:000028c0 00000028H .idata$2                CODE
 0001:000028e8 00000014H .idata$3                CODE
 0001:000028fc 000000a4H .idata$4                CODE
 0001:000029a0 00000016H .idata$6                CODE
 0001:000029c0 00000057H .edata                  CODE
 0002:00000000 000000a4H .idata$5                DATA
 0002:000000a8 00000444H .data                   DATA
 0002:00000500 00000120H .bss                    DATA

  Address         Publics by Value              Rva+Base     Lib:Object

 0000:00000000       ___safe_se_handler_table   00000000     <absolute>
 0000:00000000       ___safe_se_handler_count   00000000     <absolute>
 0001:0000001c       ??_C@_19OBNDINH@?$AAP?$AAo?$AAr?$AAt?$AA?$AA@ 1000101c     buspcie950.obj
 0001:00000028       ??_C@_1BI@IGMEDLLH@?$AA?$CF?$AAs?$AA?2?$AAU?$AAn?$AAi?$AAm?$AAo?$AAd?$AAe?$AAm?$AA?$AA@ 10001028     buspcie950.obj
 0001:00000040       ??_C@_1BK@BFIEKNFP@?$AAF?$AAr?$AAi?$AAe?$AAn?$AAd?$AAl?$AAy?$AAN?$AAa?$AAm?$AAe?$AA?$AA@ 10001040     buspcie950.obj
 0001:0000005c       ??_C@_1BG@KCOOGCNN@?$AAD?$AAe?$AAv?$AAi?$AAc?$AAe?$AAT?$AAy?$AAp?$AAe?$AA?$AA@ 1000105c     buspcie950.obj
 0001:00000074       ??_C@_1BK@HFHDBJKI@?$AAU?$AAn?$AAi?$AAm?$AAo?$AAd?$AAe?$AAm?$AA?4?$AAd?$AAl?$AAl?$AA?$AA@ 10001074     buspcie950.obj
 0001:00000090       ??_C@_19LJDFFCJJ@?$AA?$CF?$AAs?$AA?$CF?$AAs?$AA?$AA@ 10001090     buspcie950.obj
 0001:0000009c       ??_C@_1BO@DLFIJDKP@?$AA?$CF?$AAs?$AA?2?$AAS?$AAe?$AAr?$AAi?$AAa?$AAl?$AAC?$AAa?$AAb?$AAl?$AAe?$AA?$AA@ 1000109c     buspcie950.obj
 0001:000000bc       ??_C@_1O@OFBIJOJC@?$AA?$CF?$AAs?$AA?$CF?$AA0?$AA2?$AAd?$AA?$AA@ 100010bc     buspcie950.obj
 0001:000000cc       ??_C@_1CA@INOAHGHF@?$AAB?$AAu?$AAs?$AAA?$AAc?$AAc?$AAe?$AAs?$AAs?$AAH?$AAa?$AAn?$AAd?$AAl?$AAe?$AA?$AA@ 100010cc     buspcie950.obj
 0001:000000ec       ??_C@_1O@GBAEOCCH@?$AAP?$AAr?$AAe?$AAf?$AAi?$AAx?$AA?$AA@ 100010ec     buspcie950.obj
 0001:000000fc       ??_C@_1BE@GPBAGNPC@?$AAI?$AAs?$AAr?$AAH?$AAa?$AAn?$AAd?$AAl?$AAe?$AA?$AA@ 100010fc     buspcie950.obj
 0001:00000110       ??_C@_1BC@MCDIKBIL@?$AAI?$AAs?$AAt?$AAE?$AAv?$AAe?$AAn?$AAt?$AA?$AA@ 10001110     buspcie950.obj
 0001:00000124       ??_C@_1BG@LJAMCNJN@?$AAP?$AAo?$AAr?$AAt?$AAN?$AAu?$AAm?$AAb?$AAe?$AAr?$AA?$AA@ 10001124     buspcie950.obj
 0001:0000013c       ??_C@_1CC@KMPFMANC@?$AAD?$AAe?$AAv?$AAi?$AAc?$AAe?$AAA?$AAr?$AAr?$AAa?$AAy?$AAI?$AAn?$AAd?$AAe?$AAx?$AA?$AA@ 1000113c     buspcie950.obj
 0001:00000160       ??_C@_17DJMMGLBL@?$AAD?$AAl?$AAl?$AA?$AA@ 10001160     buspcie950.obj
 0001:00000168       ??_C@_19DIEFAIMH@?$AAC?$AAM?$AA?$CF?$AAd?$AA?$AA@ 10001168     buspcie950.obj
 0001:00000174       ??_C@_1M@OAJFFPML@?$AAF?$AAl?$AAa?$AAg?$AAs?$AA?$AA@ 10001174     buspcie950.obj
 0001:00000180       ??_C@_1BE@EODMIMC@?$AA?$CF?$AAs?$AA?2?$AAp?$AAo?$AAr?$AAt?$AA?$CF?$AAd?$AA?$AA@ 10001180     buspcie950.obj
 0001:00000194       ??_C@_15KOIPKGHO@?$AAC?$AAM?$AA?$AA@ 10001194     buspcie950.obj
 0001:0000019c       ??_C@_17KKLPNNMB@?$AAC?$AAO?$AAM?$AA?$AA@ 1000119c     buspcie950.obj
 0001:000001a4       ??_C@_19DINFBLAK@?$AAN?$AAa?$AAm?$AAe?$AA?$AA@ 100011a4     buspcie950.obj
 0001:000001b0       ??_C@_1CE@HBCGCCG@?$AAD?$AAr?$AAi?$AAv?$AAe?$AAr?$AAs?$AA?2?$AAA?$AAc?$AAt?$AAi?$AAv?$AAe?$AA?2?$AA?$CF?$AAs?$AA?$AA@ 100011b0     buspcie950.obj
 0001:000001d4       ??_C@_1BO@JJBEOHCE@?$AAD?$AAr?$AAi?$AAv?$AAe?$AAr?$AAs?$AA?2?$AAA?$AAc?$AAt?$AAi?$AAv?$AAe?$AA?$AA@ 100011d4     buspcie950.obj
 0001:000001f4       ??_C@_1CM@HIMBKDJM@?$AAL?$AAi?$AAn?$AAe?$AAD?$AAr?$AAi?$AAv?$AAe?$AAr?$AAD?$AAe?$AAl?$AAa?$AAy?$AAP?$AAh?$AAa?$AAs?$AAe@ 100011f4     buspcie950.obj
 0001:00000220       ??_C@_1CI@GLAIJPLJ@?$AAL?$AAi?$AAn?$AAe?$AAD?$AAr?$AAi?$AAv?$AAe?$AAr?$AAD?$AAe?$AAl?$AAa?$AAy?$AAB?$AAi?$AAt?$AAs?$AA?$AA@ 10001220     buspcie950.obj
 0001:00000248       ??_C@_1CI@OJPKJBA@?$AAB?$AAa?$AAu?$AAd?$AAr?$AAa?$AAt?$AAe?$AAM?$AAa?$AAp?$AAL?$AAi?$AAs?$AAt?$AAF?$AAr?$AAo?$AAm?$AA?$AA@ 10001248     buspcie950.obj
 0001:00000270       ??_C@_1CE@BHEKDMEI@?$AAB?$AAa?$AAu?$AAd?$AAr?$AAa?$AAt?$AAe?$AAM?$AAa?$AAp?$AAL?$AAi?$AAs?$AAt?$AAT?$AAo?$AA?$AA@ 10001270     buspcie950.obj
 0001:00000294       ??_C@_1BE@DDEHHBPD@?$AAD?$AAe?$AAv?$AAC?$AAo?$AAn?$AAf?$AAi?$AAg?$AA?$AA@ 10001294     buspcie950.obj
 0001:000002a8       ??_C@_17KNDIACFJ@?$AAT?$AAs?$AAp?$AA?$AA@ 100012a8     buspcie950.obj
 0001:000002b0       ??_C@_1BG@JDAFHBOG@?$AAI?$AAS?$AAR?$AAH?$AAa?$AAn?$AAd?$AAl?$AAe?$AAr?$AA?$AA@ 100012b0     buspcie950.obj
 0001:000002c8       ??_C@_1BG@NELPJJNN@?$AAI?$AAs?$AAr?$AAH?$AAa?$AAn?$AAd?$AAl?$AAe?$AAr?$AA?$AA@ 100012c8     buspcie950.obj
 0001:000002e0       ??_C@_1BO@KACPNJCM@?$AAi?$AAs?$AAr?$AAp?$AAc?$AAi?$AAe?$AA9?$AA5?$AA0?$AA?4?$AAd?$AAl?$AAl?$AA?$AA@ 100012e0     buspcie950.obj
 0001:00000300       ??_C@_1O@MDNCMDKF@?$AAI?$AAs?$AAr?$AAD?$AAl?$AAl?$AA?$AA@ 10001300     buspcie950.obj
 0001:00000310       ??_C@_1BO@NHAHMBJD@?$AAc?$AAo?$AAm?$AAp?$AAc?$AAi?$AAe?$AA9?$AA5?$AA0?$AA?4?$AAd?$AAl?$AAl?$AA?$AA@ 10001310     buspcie950.obj
 0001:00000330       ??_C@_1BA@CEFELOID@?$AAU?$AAa?$AAr?$AAt?$AAD?$AAl?$AAl?$AA?$AA@ 10001330     buspcie950.obj
 0001:00000340       ??_C@_1BA@BDHDGOBO@?$AAS?$AAy?$AAs?$AAI?$AAn?$AAt?$AAr?$AA?$AA@ 10001340     buspcie950.obj
 0001:00000350       ??_C@_17DJGGJCGD@?$AAI?$AAr?$AAq?$AA?$AA@ 10001350     buspcie950.obj
 0001:00000358       ??_C@_1BM@MHMIAMLB@?$AAI?$AAn?$AAt?$AAe?$AAr?$AAf?$AAa?$AAc?$AAe?$AAT?$AAy?$AAp?$AAe?$AA?$AA@ 10001358     buspcie950.obj
 0001:00000374       ??_C@_1BE@MNDDMKMB@?$AAB?$AAu?$AAs?$AAN?$AAu?$AAm?$AAb?$AAe?$AAr?$AA?$AA@ 10001374     buspcie950.obj
 0001:00000388       ??_C@_1O@LBBNFMDB@?$AAM?$AAe?$AAm?$AAL?$AAe?$AAn?$AA?$AA@ 10001388     buspcie950.obj
 0001:00000398       ??_C@_1BA@INLDIDEN@?$AAM?$AAe?$AAm?$AAB?$AAa?$AAs?$AAe?$AA?$AA@ 10001398     buspcie950.obj
 0001:000003a8       ??_C@_1M@PEPOCCHH@?$AAI?$AAo?$AAL?$AAe?$AAn?$AA?$AA@ 100013a8     buspcie950.obj
 0001:000003b4       ??_C@_1O@JMCNHCBG@?$AAI?$AAo?$AAB?$AAa?$AAs?$AAe?$AA?$AA@ 100013b4     buspcie950.obj
 0001:000003c4       ??_C@_1CE@PJBMNJAF@?$AAL?$AAi?$AAn?$AAe?$AAD?$AAr?$AAi?$AAv?$AAe?$AAr?$AAC?$AAo?$AAn?$AAt?$AAr?$AAo?$AAl?$AA?$AA@ 100013c4     buspcie950.obj
 0001:000003e8       ??_C@_1CE@HLGCKFJ@?$AAF?$AAl?$AAo?$AAw?$AAC?$AAt?$AAr?$AAl?$AAH?$AAi?$AAg?$AAh?$AAL?$AAe?$AAv?$AAe?$AAl?$AA?$AA@ 100013e8     buspcie950.obj
 0001:0000040c       ??_C@_1CC@ELLFOF@?$AAF?$AAl?$AAo?$AAw?$AAC?$AAt?$AAr?$AAl?$AAL?$AAo?$AAw?$AAL?$AAe?$AAv?$AAe?$AAl?$AA?$AA@ 1000140c     buspcie950.obj
 0001:00000430       ??_C@_1BO@MCGADMLE@?$AAR?$AAx?$AAI?$AAn?$AAt?$AAT?$AAr?$AAi?$AAg?$AAL?$AAe?$AAv?$AAe?$AAl?$AA?$AA@ 10001430     buspcie950.obj
 0001:00000450       ??_C@_1BO@ELCCHGIE@?$AAT?$AAx?$AAI?$AAn?$AAt?$AAT?$AAr?$AAi?$AAg?$AAL?$AAe?$AAv?$AAe?$AAl?$AA?$AA@ 10001450     buspcie950.obj
 0001:00000470       ??_C@_1CC@EKOCNIBB@?$AAC?$AAr?$AAy?$AAs?$AAt?$AAa?$AAl?$AAF?$AAr?$AAe?$AAq?$AAu?$AAe?$AAn?$AAc?$AAy?$AA?$AA@ 10001470     buspcie950.obj
 0001:00000494       ??_C@_1BK@KAMHHDIE@?$AAB?$AAr?$AAa?$AAn?$AAd?$AAi?$AAn?$AAg?$AAF?$AAi?$AAl?$AAe?$AA?$AA@ 10001494     buspcie950.obj
 0001:000004b0       ??_C@_1BM@CMGCPMHF@?$AAR?$AAe?$AAa?$AAd?$AAB?$AAr?$AAa?$AAn?$AAd?$AAF?$AAi?$AAl?$AAe?$AA?$AA@ 100014b0     buspcie950.obj
 0001:000004cc       ??_C@_17KACEIPNC@?$AAK?$AAe?$AAy?$AA?$AA@ 100014cc     buspcie950.obj
 0001:000004d4       ??_C@_1CK@MHPGFJDK@?$AAH?$AAa?$AAy?$AAe?$AAs?$AA?5?$AAC?$AAo?$AAm?$AAp?$AAa?$AAt?$AAi?$AAb?$AAl?$AAe?$AA?5?$AAo?$AAn?$AA?5@ 100014d4     buspcie950.obj
 0001:00000500       ??_C@_1CC@KACJOILC@?$AAS?$AAe?$AAr?$AAi?$AAa?$AAl?$AA?5?$AAC?$AAa?$AAb?$AAl?$AAe?$AA?5?$AAo?$AAn?$AA?5?$AA?$AA@ 10001500     buspcie950.obj
 0001:00000524       ??_C@_1M@FFLAJJMG@?$AA?$DM?$AAE?$AAN?$AAD?$AA?$DO?$AA?$AA@ 10001524     ConfigParser.obj
 0001:00000530       ??_C@_1CG@LGKPGFHM@?$AAN?$AAo?$AA?5?$AAC?$AAo?$AAn?$AAt?$AAr?$AAo?$AAl?$AA?5?$AA?$CI?$AAR?$AAS?$AA2?$AA3?$AA2?$AA?$CJ?$AA?$AA@ 10001530     ConfigParser.obj
 0001:00000558       ??_C@_1CO@KJKNEDLA@?$AAL?$AAo?$AAw?$AA?5?$AAE?$AAn?$AAa?$AAb?$AAl?$AAe?$AA?5?$AA?$CI?$AAR?$AAS?$AA4?$AA2?$AA2?$AA?1?$AA4?$AA8@ 10001558     ConfigParser.obj
 0001:00000588       ??_C@_1BI@LGOMGNKN@?$AAH?$AAi?$AAg?$AAh?$AA?5?$AAE?$AAn?$AAa?$AAb?$AAl?$AAe?$AA?$AA@ 10001588     ConfigParser.obj
 0001:000005a0       ??_C@_19BIEPDBPA@?$AAT?$AAy?$AAp?$AAe?$AA?$AA@ 100015a0     ConfigParser.obj
 0001:000005ac       ??_C@_1BK@CENGCIFF@?$AAT?$AAo?$AA_?$AAB?$AAa?$AAu?$AAd?$AA_?$AAR?$AAa?$AAt?$AAe?$AA?$AA@ 100015ac     ConfigParser.obj
 0001:000005c8       ??_C@_1BO@CILDMCD@?$AAF?$AAr?$AAo?$AAm?$AA_?$AAB?$AAa?$AAu?$AAd?$AA_?$AAR?$AAa?$AAt?$AAe?$AA?$AA@ 100015c8     ConfigParser.obj
 0001:000005e8       ??_C@_1BE@GELDBLFK@?$AAT?$AAa?$AAb?$AA_?$AAA?$AAb?$AAo?$AAu?$AAt?$AA?$AA@ 100015e8     ConfigParser.obj
 0001:000005fc       ??_C@_1DA@NCKAKAMN@?$AAT?$AAa?$AAb?$AA_?$AAL?$AAi?$AAn?$AAe?$AA_?$AAD?$AAr?$AAi?$AAv?$AAe?$AAr?$AA_?$AAC?$AAo?$AAn?$AAt@ 100015fc     ConfigParser.obj
 0001:0000062c       ??_C@_1CA@LJNFGPHD@?$AAT?$AAa?$AAb?$AA_?$AAF?$AAi?$AAf?$AAo?$AA_?$AAL?$AAe?$AAv?$AAe?$AAl?$AAs?$AA?$AA@ 1000162c     ConfigParser.obj
 0001:0000064c       ??_C@_1CK@NLOLPFMM@?$AAT?$AAa?$AAb?$AA_?$AAB?$AAa?$AAu?$AAd?$AAr?$AAa?$AAt?$AAe?$AA_?$AAM?$AAa?$AAp?$AAp?$AAi?$AAn?$AAg@ 1000164c     ConfigParser.obj
 0001:00000678       ??_C@_1CM@OFMOCLCD@?$AAT?$AAa?$AAb?$AA_?$AAC?$AAr?$AAy?$AAs?$AAt?$AAa?$AAl?$AA_?$AAF?$AAr?$AAe?$AAq?$AAu?$AAe?$AAn?$AAc@ 10001678     ConfigParser.obj
 0001:000006a4       ??_C@_1DG@MMINKBLM@?$AAF?$AAl?$AAo?$AAw?$AA_?$AAC?$AAo?$AAn?$AAt?$AAr?$AAo?$AAl?$AA_?$AAO?$AAf?$AAf?$AA_?$AAL?$AAe?$AAv@ 100016a4     ConfigParser.obj
 0001:000006dc       ??_C@_1DG@FFKMCLJC@?$AAF?$AAl?$AAo?$AAw?$AA_?$AAC?$AAo?$AAn?$AAt?$AAr?$AAo?$AAl?$AA_?$AAO?$AAf?$AAf?$AA_?$AAL?$AAe?$AAv@ 100016dc     ConfigParser.obj
 0001:00000714       ??_C@_1DE@JAENBBJL@?$AAF?$AAl?$AAo?$AAw?$AA_?$AAC?$AAo?$AAn?$AAt?$AAr?$AAo?$AAl?$AA_?$AAO?$AAn?$AA_?$AAL?$AAe?$AAv?$AAe@ 10001714     ConfigParser.obj
 0001:00000748       ??_C@_1DE@JGMJLLF@?$AAF?$AAl?$AAo?$AAw?$AA_?$AAC?$AAo?$AAn?$AAt?$AAr?$AAo?$AAl?$AA_?$AAO?$AAn?$AA_?$AAL?$AAe?$AAv?$AAe@ 10001748     ConfigParser.obj
 0001:0000077c       ??_C@_1DO@FFHHIFI@?$AAR?$AAx?$AA_?$AAI?$AAn?$AAt?$AAe?$AAr?$AAr?$AAu?$AAp?$AAt?$AA_?$AAT?$AAr?$AAi?$AAg?$AAg?$AAe?$AAr@ 1000177c     ConfigParser.obj
 0001:000007bc       ??_C@_1DO@JMHGPCHG@?$AAR?$AAx?$AA_?$AAI?$AAn?$AAt?$AAe?$AAr?$AAr?$AAu?$AAp?$AAt?$AA_?$AAT?$AAr?$AAi?$AAg?$AAg?$AAe?$AAr@ 100017bc     ConfigParser.obj
 0001:000007fc       ??_C@_1DO@HONDFPK@?$AAT?$AAx?$AA_?$AAI?$AAn?$AAt?$AAe?$AAr?$AAr?$AAu?$AAp?$AAt?$AA_?$AAT?$AAr?$AAi?$AAg?$AAg?$AAe?$AAr@ 100017fc     ConfigParser.obj
 0001:0000083c       ??_C@_1DO@JOMMLPNE@?$AAT?$AAx?$AA_?$AAI?$AAn?$AAt?$AAe?$AAr?$AAr?$AAu?$AAp?$AAt?$AA_?$AAT?$AAr?$AAi?$AAg?$AAg?$AAe?$AAr@ 1000183c     ConfigParser.obj
 0001:0000087c       ??_C@_1BO@CLLBHNOO@?$AAF?$AAl?$AAo?$AAw?$AA_?$AAO?$AAf?$AAf?$AA_?$AAL?$AAe?$AAv?$AAe?$AAl?$AA?$AA@ 1000187c     ConfigParser.obj
 0001:0000089c       ??_C@_1BM@FKEALHLG@?$AAF?$AAl?$AAo?$AAw?$AA_?$AAO?$AAn?$AA_?$AAL?$AAe?$AAv?$AAe?$AAl?$AA?$AA@ 1000189c     ConfigParser.obj
 0001:000008b8       ??_C@_1EA@FCDBIJCN@?$AAR?$AAe?$AAc?$AAe?$AAi?$AAv?$AAe?$AA_?$AAI?$AAn?$AAt?$AAe?$AAr?$AAr?$AAu?$AAp?$AAt?$AA_?$AAT?$AAr@ 100018b8     ConfigParser.obj
 0001:000008f8       ??_C@_1EC@JOHHNGND@?$AAT?$AAr?$AAa?$AAn?$AAs?$AAm?$AAi?$AAt?$AA_?$AAI?$AAn?$AAt?$AAe?$AAr?$AAr?$AAu?$AAp?$AAt?$AA_?$AAT@ 100018f8     ConfigParser.obj
 0001:0000093c       ??_C@_1M@MNHBCACD@?$AAT?$AAi?$AAt?$AAl?$AAe?$AA?$AA@ 1000193c     ConfigParser.obj
 0001:00000948       ??_C@_1CI@IMABDCBP@?$AAL?$AAi?$AAn?$AAe?$AA_?$AAD?$AAr?$AAi?$AAv?$AAe?$AAr?$AA_?$AAC?$AAo?$AAn?$AAt?$AAr?$AAo?$AAl?$AA?$AA@ 10001948     ConfigParser.obj
 0001:00000970       ??_C@_1CC@FHAFLLA@?$AAB?$AAa?$AAu?$AAd?$AAr?$AAa?$AAt?$AAe?$AA_?$AAM?$AAa?$AAp?$AAp?$AAi?$AAn?$AAg?$AA?$AA@ 10001970     ConfigParser.obj
 0001:00000994       ??_C@_1BI@LMBHJBLG@?$AAT?$AAa?$AAb?$AA_?$AAO?$AAp?$AAt?$AAi?$AAo?$AAn?$AAs?$AA?$AA@ 10001994     ConfigParser.obj
 0001:000009ac       ??_C@_1BI@GEBICGMH@?$AAF?$AAi?$AAf?$AAo?$AA_?$AAL?$AAe?$AAv?$AAe?$AAl?$AAs?$AA?$AA@ 100019ac     ConfigParser.obj
 0001:000009c4       ??_C@_1CE@FHCKENKN@?$AAC?$AAr?$AAy?$AAs?$AAt?$AAa?$AAl?$AA_?$AAF?$AAr?$AAe?$AAq?$AAu?$AAe?$AAn?$AAc?$AAy?$AA?$AA@ 100019c4     ConfigParser.obj
 0001:000009e8       ??_C@_1CE@EOJPOKCA@?$AAA?$AAp?$AAp?$AAl?$AAi?$AAc?$AAa?$AAt?$AAi?$AAo?$AAn?$AA_?$AAT?$AAi?$AAt?$AAl?$AAe?$AA?$AA@ 100019e8     ConfigParser.obj
 0001:00000a0c       ??_C@_15GANGMFKL@?$AA?$CF?$AAs?$AA?$AA@ 10001a0c     ConfigParser.obj
 0001:00000a14       ??_C@_15JJPIMNBO@?$AAr?$AAb?$AA?$AA@ 10001a14     ConfigParser.obj
 0001:00000a1c       ??_C@_1BI@MHELFDAB@?$AA?2?$AAW?$AAi?$AAn?$AAd?$AAo?$AAw?$AAs?$AA?2?$AA?$CF?$AAs?$AA?$AA@ 10001a1c     ConfigParser.obj
 0001:00000a8e       _KLibFreeShareMem          10001a8e f i buspcie950.obj
 0001:00000aab       _DllEntry                  10001aab f   buspcie950.obj
 0001:00000b43       _GetBrandingData           10001b43 f   buspcie950.obj
 0001:00000b59       _Deinit                    10001b59 f   buspcie950.obj
 0001:00000d01       _Init                      10001d01 f   buspcie950.obj
 0001:00001dc6       __tfsubstring              10002dc6 f   ConfigParser.obj
 0001:00001e00       ?_ffeosubsec@@YAHPAXQAG@Z  10002e00 f   ConfigParser.obj
 0001:00001e38       _InitializeConfigInfo      10002e38 f   ConfigParser.obj
 0001:00001e7e       ?ValidateCrystalFrequency@@YAHH@Z 10002e7e f   ConfigParser.obj
 0001:00001f2a       ?ValidateValues@@YAXPAU_CONFIG_DATA_@@@Z 10002f2a f   ConfigParser.obj
 0001:00002055       ?_textractValue@@YAPAGPAG@Z 10003055 f   ConfigParser.obj
 0001:00002084       _ParseConfigFile           10003084 f   ConfigParser.obj
 0001:00002810       _BusTransBusAddrToStatic   10003810 f   ceddk:CEDDK.dll
 0001:00002816       _BusTransBusAddrToVirtual  10003816 f   ceddk:CEDDK.dll
 0001:0000281c       _CreateBusAccessHandle     1000381c f   ceddk:CEDDK.dll
 0001:00002822       _KernelLibIoControl        10003822 f   coredll:COREDLL.dll
 0001:00002828       _EventModify               10003828 f   coredll:COREDLL.dll
 0001:0000282e       _InterruptDone             1000382e f   coredll:COREDLL.dll
 0001:00002834       _DeactivateDevice          10003834 f   coredll:COREDLL.dll
 0001:0000283a       _wcstoul                   1000383a f   coredll:COREDLL.dll
 0001:00002840       _wcslen                    10003840 f   coredll:COREDLL.dll
 0001:00002846       _ActivateDeviceEx          10003846 f   coredll:COREDLL.dll
 0001:0000284c       _CreateThread              1000384c f   coredll:COREDLL.dll
 0001:00002852       _InterruptInitialize       10003852 f   coredll:COREDLL.dll
 0001:00002858       _LoadIntChainHandler       10003858 f   coredll:COREDLL.dll
 0001:0000285e       _wcschr                    1000385e f   coredll:COREDLL.dll
 0001:00002864       _wcsstr                    10003864 f   coredll:COREDLL.dll
 0001:0000286a       _wsprintfW                 1000386a f   coredll:COREDLL.dll
 0001:00002870       _free                      10003870 f   coredll:COREDLL.dll
 0001:00002876       _malloc                    10003876 f   coredll:COREDLL.dll
 0001:0000287c       _wcstol                    1000387c f   coredll:COREDLL.dll
 0001:00002882       _wcscpy                    10003882 f   coredll:COREDLL.dll
 0001:00002888       __chkstk                   10003888 f   coredll:COREDLL.dll
 0001:0000288e       _wcscmp                    1000388e f   coredll:COREDLL.dll
 0001:00002894       _fgetws                    10003894 f   coredll:COREDLL.dll
 0001:0000289a       _wcsrchr                   1000389a f   coredll:COREDLL.dll
 0001:000028a0       _fclose                    100038a0 f   coredll:COREDLL.dll
 0001:000028a6       __wtol                     100038a6 f   coredll:COREDLL.dll
 0001:000028ac       _feof                      100038ac f   coredll:COREDLL.dll
 0001:000028b2       __wfopen                   100038b2 f   coredll:COREDLL.dll
 0001:000028b8       _swprintf                  100038b8 f   coredll:COREDLL.dll
 0001:000028c0       __IMPORT_DESCRIPTOR_CEDDK  100038c0     ceddk:CEDDK.dll
 0001:000028d4       __IMPORT_DESCRIPTOR_COREDLL 100038d4     coredll:COREDLL.dll
 0001:000028e8       __NULL_IMPORT_DESCRIPTOR   100038e8     ceddk:CEDDK.dll
 0002:00000000       __imp__BusTransBusAddrToVirtual 10004000     ceddk:CEDDK.dll
 0002:00000004       __imp__CreateBusAccessHandle 10004004     ceddk:CEDDK.dll
 0002:00000008       __imp__BusTransBusAddrToStatic 10004008     ceddk:CEDDK.dll
 0002:0000000c       \177CEDDK_NULL_THUNK_DATA  1000400c     ceddk:CEDDK.dll
 0002:00000010       __imp__KernelLibIoControl  10004010     coredll:COREDLL.dll
 0002:00000014       __imp__EventModify         10004014     coredll:COREDLL.dll
 0002:00000018       __imp__DisableThreadLibraryCalls 10004018     coredll:COREDLL.dll
 0002:0000001c       __imp__InterruptDone       1000401c     coredll:COREDLL.dll
 0002:00000020       __imp__WaitForSingleObject 10004020     coredll:COREDLL.dll
 0002:00000024       __imp__CloseHandle         10004024     coredll:COREDLL.dll
 0002:00000028       __imp__DeactivateDevice    10004028     coredll:COREDLL.dll
 0002:0000002c       __imp__wcstoul             1000402c     coredll:COREDLL.dll
 0002:00000030       __imp__RegQueryValueExW    10004030     coredll:COREDLL.dll
 0002:00000034       __imp__RegSetValueExW      10004034     coredll:COREDLL.dll
 0002:00000038       __imp__wcslen              10004038     coredll:COREDLL.dll
 0002:0000003c       __imp__ActivateDeviceEx    1000403c     coredll:COREDLL.dll
 0002:00000040       __imp__RegCreateKeyExW     10004040     coredll:COREDLL.dll
 0002:00000044       __imp__CreateThread        10004044     coredll:COREDLL.dll
 0002:00000048       __imp__InterruptInitialize 10004048     coredll:COREDLL.dll
 0002:0000004c       __imp__CreateEventW        1000404c     coredll:COREDLL.dll
 0002:00000050       __imp__LoadIntChainHandler 10004050     coredll:COREDLL.dll
 0002:00000054       __imp__wcschr              10004054     coredll:COREDLL.dll
 0002:00000058       __imp__wcsstr              10004058     coredll:COREDLL.dll
 0002:0000005c       __imp__wsprintfW           1000405c     coredll:COREDLL.dll
 0002:00000060       __imp__RegEnumKeyExW       10004060     coredll:COREDLL.dll
 0002:00000064       __imp__RegCloseKey         10004064     coredll:COREDLL.dll
 0002:00000068       __imp__free                10004068     coredll:COREDLL.dll
 0002:0000006c       __imp__malloc              1000406c     coredll:COREDLL.dll
 0002:00000070       __imp__wcstol              10004070     coredll:COREDLL.dll
 0002:00000074       __imp__wcscpy              10004074     coredll:COREDLL.dll
 0002:00000078       __imp__RegOpenKeyExW       10004078     coredll:COREDLL.dll
 0002:0000007c       __imp___chkstk             1000407c     coredll:COREDLL.dll
 0002:00000080       __imp__wcscmp              10004080     coredll:COREDLL.dll
 0002:00000084       __imp__fgetws              10004084     coredll:COREDLL.dll
 0002:00000088       __imp__wcsrchr             10004088     coredll:COREDLL.dll
 0002:0000008c       __imp__fclose              1000408c     coredll:COREDLL.dll
 0002:00000090       __imp___wtol               10004090     coredll:COREDLL.dll
 0002:00000094       __imp__feof                10004094     coredll:COREDLL.dll
 0002:00000098       __imp___wfopen             10004098     coredll:COREDLL.dll
 0002:0000009c       __imp__swprintf            1000409c     coredll:COREDLL.dll
 0002:000000a0       \177COREDLL_NULL_THUNK_DATA 100040a0     coredll:COREDLL.dll
 0002:000000a8       _dpCurSettings             100040a8     buspcie950.obj
 0002:00000500       _m_pDispatchThread         10004500     buspcie950.obj
 0002:00000580       _Pcie950BusInfo            10004580     <common>

 entry point at        0001:00000aab

 Static symbols

 0001:00000ac1       _BusIstThread              10001ac1 f   buspcie950.obj
 0001:00000bd3       _ReadKeyList               10001bd3 f   buspcie950.obj
 0001:00000c73       _ReadKeyDword              10001c73 f   buspcie950.obj
 0001:00000cb2       _WriteKeyDword             10001cb2 f   buspcie950.obj
 0001:00000cd4       _WriteKeyString            10001cd4 f   buspcie950.obj
